:1000000008F30720E90000000F01000011010000C3
:10001000130100001501000017010000B006F8DF11
:1000200000000000000000000000000019010000B6
:100030001B010000000000001D01000071370000DE
:1000400021010000210100004539000021010000CC
:100050002101000021010000210100002101000018
:100060002101000021010000210100002101000008
:1000700021010000210100002101000021010000F8
:1000800021010000210100002101000021010000E8
:1000900021010000210100002101000021010000D8
:1000A000553D000021010000210100002101000058
:1000B00021010000210100002101000021010000B8
:1000C000210100002101000021010000DFF80CD017
:1000D00000F072F800480047B551000008F307200F
:1000E000D0F800D0D0F804F04FF080500D494FF018
:1000F000000240F8042B8842FBD10B480B494FF01B
:10010000000240F8042B8842FBD109480047FEE773
:10011000FEE7FEE7FEE7FEE7FEE7FEE7FEE7FEE7B7
:10012000FEE700000080001000C00720004008200B
:10013000CD00000010B50B4604461146184600F0ED
:1001400027F8C4E9000110BD40EA01039B0703D072
:1001500009E008C9121F08C0042AFAD203E011F806
:10016000013B00F8013B521EF9D27047D2B201E0C8
:1001700000F8012B491EFBD270470022F6E710B5AC
:1001800013460A4604461946FFF7F0FF204610BD05
:1001900070B500242546002801DA012440420029D8
:1001A00001DA0125494200F019F8AC4200D0404282
:1001B000002C00D0494270BD064C074D06E0E068B7
:1001C00040F0010394E8070098471034AC42F6D39E
:1001D000FFF780FFB45D0000E45D000030B50B4622
:1001E000014600202022012409E021FA02F59D4267
:1001F00005D303FA02F5491B04FA02F52844151E3B
:10020000A2F10102F1DC30BD30B58C1810F8012BE1
:1002100012F00F0301D110F8013B120906D110F8BA
:10022000012B03E010F8015B01F8015B5B1EF9D1C3
:1002300001E001F8013B521EFBD1A142E6D30020B0
:1002400030BD000010B5044600F016F80848005D07
:1002500040F09071074801604468002CFCDA4FF4CC
:100260000011016000F016F84FF6F070204010BD4C
:10027000D45C0000004003400549486828B9EFF30A
:10028000108202F0010272B68A60401C486070471A
:1002900040C107200549486810B1401E486003D19D
:1002A0008868002800D162B67047000040C107206E
:1002B0007047000010B5044C0022626000F058F84E
:1002C00060680028FCD110BD4CC1072070B5002328
:1002D000084D0AE0CE5C04885B1C86EA14269BB2BB
:1002E00035F8166086EA04240480521E92B2F1D2D8
:1002F00070BD0000C057000000207047FFFFFFFFE7
:100300001648022141600021816001670B22C26012
:10031000032242614EF66022826101224260104A4D
:10032000182082F800040420921EC2F800010D4833
:10033000C26822F44052C260C26C22F4405242F4BD
:100340000052C26408484FF48002C263026A42F459
:100350008002026205484160002070470080004032
:1003600002E000E000C0024000C009204CC10720AC
:1003700041F28832904225D8642800D210BB42F264
:10038000107291421ED805291CD3E8B1144B5A684B
:10039000002AFCD1B0B1134AB2FBF0F24FF47A70EC
:1003A0004143B1FBF2F058600F4802214160002147
:1003B000816001670B21C1600321416151088161A6
:1003C00001214160002070470848826801EB410329
:1003D000C3EBC11183689B1AB3EBC10FFAD3F1E7EA
:1003E0004CC1072040420F0000800040000009403F
:1003F00001460007C00E090600D5401C704704F0F6
:1004000001BD70474D0B00002DE9FC41074600205F
:1004100090460E46ADF8000004460EE0351B402D18
:1004200000D9402539192A460D4800F059FBAAB2D7
:100430000B496846FFF74AFF2C44B442EED3391902
:10044000424601A800F04CFBBDF80000BDF80410C6
:10045000884202D10120BDE8FC810020FBE70000BA
:10046000F9DB07202DE9F041664C002788B0A77022
:10047000E770DFF894814FF40056277101251922A7
:10048000314601A800F02CFB022216213046FFF76E
:10049000BBFF00287ED0DDF81210022206F1190001
:1004A000FFF7B2FF002875D09DF8040006282AD275
:1004B000DFE800F02A03032A2A1CD8F87410DDF8BC
:1004C0000E30491C8B421ED2D8F87420DDF80E3055
:1004D000D21ADDF81230521C9A4214D3DDF80E20E5
:1004E000DDF812301A448A420DD80DE0DDF8121002
:1004F000B1F5F42F00D9A570DDF81610C1F30B414A
:10050000B1F5C87F00D0A570012803D0022801D022
:10051000052839D1022206F21D416846009700F0F5
:10052000DFFA0099029889B2884200D0A5700122B2
:1005300006F225416846009700F0D2FA0099BDF80E
:100540000500C9B2884200D0A5709DF804000228B9
:100550001AD1042206F249416846009700F0C0FA19
:10056000DDF816000099884200D0A570012206F23D
:100570004D416846009700F0B3FA00989DF80710C7
:10058000C0B2814200D0A5709DF81C00401EFE281C
:1005900002D200E01EE0A570BDF80500A0F57F4185
:1005A000FF3901D0482802D19DF8070020B901A8E1
:1005B00000F074FA00B9A570DDF812001B3606448D
:1005C00001A800F06BFA30B1E07880B1217988425F
:1005D0000DD012E0A5709DF81C0010B92079401CC8
:1005E0002071E078401CC0B2E0700C2801D3A570E7
:1005F00003E0A07800283FF442AFA07808B0BDE83F
:10060000F0810000BCC00720785B000070B500F0EE
:1006100049F81049104D114E114C087050B1114954
:1006200000EBC00001EB800080688047000609D520
:10063000206870BD822020602120286078463060CC
:10064000822070BD00202060286078463060002045
:1006500070BD00005CC1072070C0072074C0072077
:100660006CC00720DC5C00000948007828B109490B
:1006700000EBC00051F820000047074982200860C5
:1006800006492120086078460549086082207047A5
:100690005CC10720DC5C00006CC0072070C0072034
:1006A00074C0072070B5002400BF00BF00BF00BFAA
:1006B00000BF00BF00BF00BF00BF00BF00BF00BF42
:1006C00000BF00BF00BF00BF00BF00BF00BF00BF32
:1006D00000BF00BF00BF00BF00BF00BF00BF00BF22
:1006E00000BF00BF00BF00BF2D4E4FF08055F56327
:1006F0009F2001F059FC002001F056FC60F3070434
:10070000002001F051FC60F30F24002001F04CFCAC
:1007100060F31744B56300BF00BF00BF00BF00BF58
:1007200000BF00BF00BF00BF00BF00BF00BF00BFD1
:1007300000BF00BF00BF00BF00BF00BF00BF00BFC1
:1007400000BF00BF00BF00BF00BF00BF00BF00BFB1
:1007500000BF00BF00BF1349601A8C421AD00BDCE7
:10076000A4F1C204B4F5A11414D0B4F5803F11D0A3
:10077000B4F5003F0BD10DE00B49401805D00B49F3
:10078000401809D00A49C84201D1022400E00024DF
:10079000204670BD0324FBE7042402F0A9FCF7E720
:1007A00000C00920C220180003FBD6FF00FFFEFF97
:1007B0000001F8FF054982200860054922200860F1
:1007C0007846044908608220704700006CC007200A
:1007D00070C0072074C007200549822008600549C1
:1007E0002120086078460449086082207047000094
:1007F0006CC0072070C0072074C007200549822004
:100800000860054922200860784604490860822073
:10081000704700006CC0072070C0072074C007201C
:100820002DE9F041144B154D154E1B78154C63B155
:100830009AB1154F03EBC30307EB83031B6998477A
:10084000000612D52068BDE8F081822020602120BA
:100850002860784630608220F5E7862020600920F5
:100860002860784630608620EDE700202060286010
:10087000784630600020E6E75CC1072070C00720A2
:1008800074C007206CC00720DC5C00002DE9F0413B
:10089000144B154D154E1B78154C63B19AB1154F7D
:1008A00003EBC30307EB83039B699847000612D54C
:1008B0002068BDE8F08182202060222028607846F0
:1008C00030608220F5E78620206009202860784685
:1008D00030608620EDE70020206028607846306098
:1008E0000020E6E75CC1072070C0072074C0072025
:1008F0006CC00720DC5C0000F8B5184C184D194E90
:100900002778194CDDF818C087B1BCF1000F15D05D
:10091000CDF800C0DFF854C007EBC7070CEB870722
:10092000FF69B847000611D52068F8BD8220206015
:1009300022202860784630608220F8BD8620206022
:1009400009202860784630608620F8BD00202060AD
:100950002860784630600020F8BD00005CC10720A8
:1009600070C0072074C007206CC00720DC5C00004A
:1009700070B50948022400F11F05816829B1007B88
:10098000000607D4022003F0C5FC2C7300F06EFBB8
:10099000002070BD012070BDC1DB072010B50C48E0
:1009A0000C4C8068A178884200D2A0700849A278D7
:1009B0004039822003F0DEFC032060700448A278F6
:1009C0001F308168891A81600021017310BD000009
:1009D000C1DB072078C007202DE9F04113A000F00B
:1009E00069F8154800264FF47A770670C821384612
:1009F000FFF760FC114CA06842F21075A168091A5B
:100A0000A942FBD3C8213846FFF754FCA068A1686F
:100A1000091AA942FBD3C8213846FFF74BFC084806
:100A2000022186708171C670BDE8F08146494C454F
:100A3000204572720000000068C0072000000940D5
:100A4000BCC0072070B5002510240220FFF7FAFB78
:100A5000C0F30B100544641EF7D129094FF47A70D6
:100A6000B1FBF0F06422B1FBF2F10A22B1FBF2F328
:100A700002FB1311000741EA1060132800D118206F
:100A80000149086070BD000040C1072002480068AD
:100A900040F0C8707047000040C107200021425C50
:100AA00012B9491C1829FAD3182901D0002070471F
:100AB0000120704770B505460024204604F06AFB0B
:100AC000002801DA601E70BD285D0028FBD004F00C
:100AD00087FA002802DB641CE4B2F5E7002070BD51
:100AE00010B50B46014600241846FFF799FE204634
:100AF00010BD00000E4810B54178022908D0032926
:100B00000ED0042910D0052901D10021417010BD5B
:100B10000848C07B2828FAD1BDE8104000F034B95D
:100B2000BDE8104000F0A2BA822003F0F3FBF7E723
:100B300078C00720C1DB072010B51449022003F05C
:100B4000F3F913498870487860B101280ED002206B
:100B500003F0E0FB0D4902205F310873BDE810404F
:100B600000F084BABDE8104000F014B807484030E7
:100B7000C07B2A2805D02F2807D1BDE8104000F0FF
:100B800035B9BDE8104000F075B910BD81DB072014
:100B900078C007202DE9F0414A4D4B4C0021A87840
:100BA000A4F1400202E0535C6354491C03468142B5
:100BB000F9D31F2B7CD120684449884278D1424E1A
:100BC00060681F364FF001087060A068B060607BFD
:100BD00018B9A07B08B1102802D986F80C8063E010
:100BE000E07B1E28F9D011DC122833D006DC68B374
:100BF0000328F2D1BDE8F04100F00EBA1528ECD080
:100C00001A28EAD1BDE8F04100F07EB902272A286F
:100C10002ED011DC232821D0252823D02828DCD170
:100C200000F08AF900282CD0207B00061ED56F70BA
:100C3000BDE8F04100F0A8B82F2824D05528CCD02A
:100C40005A28CAD1BDE8F04100F042B9BDE8F041F0
:100C500000F01EBABDE8F04100F03AB8BDE8F0413E
:100C600000F0B4B9BDE8F04100F08EB9022018E000
:100C700000F062F9002804D0207B000610D485F82B
:100C80000180BDE8F08100F057F90028F9D0207B01
:100C9000000605D485F80180C5F82880F1E707E053
:100CA000822003F037FB3773BDE8F04100F0DEB976
:100CB000822003F02FFB022003F02CFB062068703B
:100CC000DFE7000078C00720C1DB0720555342430F
:100CD0001CB5FFF74DFE00284ED028480A220621F9
:100CE0000388684604F06AFC2548002280230270CD
:100CF000437082700121C1702021017143718271A2
:100D0000C27141220272542242724F2282724C22DC
:100D1000C272017341738173C173462202745023FE
:100D20004374722383746923C3746E23037574231D
:100D300043758175C2756C220276612242767322F8
:100D400082766822C276017741778177C1779DF8F4
:100D5000011080F820109DF8021080F821109DF8F5
:100D6000031080F822109DF8041080F82310054924
:100D700024208870FFF712FE1CBD00000404000050
:100D800081DB072078C0072070B5154D2C6B402CF7
:100D900000D94024E86AE96902198A4202D90C1A8A
:100DA00004216970214604F03DFB22460D49822052
:100DB00003F0E0FAE86A2044E862286B011B0A4865
:100DC00029638268A2EB0402826005D06978022957
:100DD00001D00021017370BD03216970F9E70000A3
:100DE00078C00720F9DB0720E0DB07202DE9F04180
:100DF0001D4CA178E06A4218E1698A4206D9081AB6
:100E0000A07005206070022003F084FA0021A07811
:100E1000164B174DE26A08E056186F5C9E5DBE42A5
:100E200002D00021A16202E0491C8142F4D31118D2
:100E3000E162216B0A1A0E49226301F15F018B689E
:100E4000A3EB0000886002D06078052809D1A06A71
:100E500028B100200873BDE8F04100F007B9012077
:100E6000F8E7BDE8F081000078C00720F9DB072033
:100E700081DB072010B5144CA178E06A4218E169C3
:100E80008A4206D9081AA07005206070022003F07B
:100E900041FAA178E06A04F00BFBA178E06A08440B
:100EA000E062206B421A094822638368A3EB0101C8
:100EB000816002D06178052905D100210173BDE868
:100EC000104000F0D3B810BD78C00720E0DB072049
:100ED00010B5FFF74DFD002811D00948002106226A
:100EE000017042708170C170017141718171C17175
:100EF000044908208870BDE81040FFF74FBD10BDC1
:100F000081DB072078C0072010B5FFF731FD0028EE
:100F10000DD0074803210170002141708170C1701C
:100F2000044904208870BDE81040FFF737BD10BDAC
:100F300081DB072078C00720114810B5D0F81110C8
:100F4000027D09BA21F0FF0111430E4A4902D16224
:100F5000C18A49BA49021163806888420DD0822053
:100F600003F0D8F9022003F0D5F9054902201F311A
:100F7000087300F07BF8002010BD012010BD0000B8
:100F8000C1DB072078C0072010B5FFF7F1FC00286F
:100F900016D00C4A0C48116A491E0B0E03700B0C3C
:100FA00043700B0A8370C1700021017141710223EB
:100FB0008371C17108209070BDE81040FFF7EEBC4E
:100FC00010BD000078C0072081DB072010B5FFF7B7
:100FD000CFFC00281AD00E4800210E4B0170417042
:100FE00081700822C2701A6A140E0471140C4471C4
:100FF000140A8471C2710222027241728272C17239
:101000000C209870BDE81040FFF7C8BC10BD000070
:1010100081DB072078C0072010B5FFF7A9FC002866
:101020001FD010487021022201700021417082708F
:10103000C1700171417181710A22C27101724172E4
:101040008172C17230220273012242738173C173B3
:1010500001744174044912208870BDE81040FFF704
:101060009DBC10BD81DB072078C00720064910B564
:10107000044808600D22822003F07CF90349052012
:10108000487010BD55534253E0DB072078C007205D
:10109000094810B5816839B1007B000601D582206E
:1010A00000E0022003F036F9034900201F310873E5
:1010B000BDE81040FFF7DABFC1DB07202DE9FC5F78
:1010C0008846044601A9414800F0C4FA404D414E0B
:1010D000414FE0BB03208DF8000020098DF801008E
:1010E00020018DF802004FF000098DF8039000BF39
:1010F00000BF00BF00BF00BF00BF00BF00BF00BFF8
:1011000000BF00BF00BF00BF00BF00BF00BF00BFE7
:1011100000BF00BF00BF00BF00BF00BF00BF00BFD7
:1011200000BF00BF00BF00BF00BF00BF00BFDFF8AF
:10113000ACB04FF0805ACBF83CA00421684600F0D8
:101140003DFF0024002000F02FFFC0B200E005E0CA
:101150008DF8040018F80410884208D08220286016
:1011600022203060784638608220BDE8FC9F641CF5
:10117000B4F5805FE6D3CBF838A000BF00BF00BF56
:1011800000BF00BF00BF00BF00BF00BF00BF00BF67
:1011900000BF00BF00BF00BF00BF00BF00BF00BF57
:1011A00000BF00BF00BF00BF00BF00BF00BF00BF47
:1011B00000BF00BF00BF00BF00BFC5F80090784669
:1011C000C6F8009038600020CFE70000A08601003C
:1011D0006CC0072070C0072074C0072000C0092021
:1011E0002DE9F0474FF0000900BF00BF00BF00BF6E
:1011F00000BF00BF00BF00BF00BF00BF00BF00BFF7
:1012000000BF00BF00BF00BF00BF00BF00BF00BFE6
:1012100000BF00BF00BF00BF00BF00BF00BF00BFD6
:1012200000BF00BF00BF00BF344E4FF08055F563D4
:101230009F2000F0B9FE002000F0B6FE00F0FF088D
:10124000002000F0B1FEC4B2002000F0ADFEC1B23B
:10125000B56300BF00BF00BF00BF00BF00BF00BF3D
:1012600000BF00BF00BF00BF00BF00BF00BF00BF86
:1012700000BF00BF00BF00BF00BF00BF00BF00BF76
:1012800000BF00BF00BF00BF00BF00BF00BF00BF66
:1012900000BF1B4D1B4E1C4FB8F1C20F01D1202CBB
:1012A00008D0822028602120306078463860822073
:1012B000BDE8F0871548142912D0152913D0162936
:1012C00015D0182916D0C0F80090002000F0D2F8F0
:1012D000C5F800907846C6F8009038600020E7E72F
:1012E0004FF4801101E04FF400110160EDE74FF47D
:1012F0008001FAE74FF08071F7E7000000C0092095
:101300006CC0072070C0072074C0072054C107209C
:101310002DE9F04FDFF89480DFF894B089B00F002A
:1013200004464FF0000628D04FF4805501462A4667
:101330006846FEF7FFFEDDE900A105912A46214639
:1013400006A8FEF7F7FEDDE906404FF00009BD1BD9
:10135000C0F58051A94200D20D4620B1544517D1A5
:101360000599884214D1204600F09AFF00060FD557
:10137000D8F8000009B0BDE8F08F8621C8F8001049
:101380000921CBF8001079460A4801608620F1E770
:101390002E44641C4846BE42D9D3C8F800007946A2
:1013A000CBF80000034801600020E3E76CC0072091
:1013B00070C0072074C007204FF4805070470000B1
:1013C000014800687047000054C1072070B504460A
:1013D00000BF00BF00BF00BF00BF00BF00BF00BF15
:1013E00000BF00BF00BF00BF00BF00BF00BF00BF05
:1013F00000BF00BF00BF00BF00BF00BF00BF00BFF5
:1014000000BF00BF00BF00BF00BF00BF00BF00BFE4
:10141000174E4FF08055F563052000F0C5FD002004
:1014200000F0C2FD2070B56300BF00BF00BF00BF69
:1014300000BF00BF00BF00BF00BF00BF00BF00BFB4
:1014400000BF00BF00BF00BF00BF00BF00BF00BFA4
:1014500000BF00BF00BF00BF00BF00BF00BF00BF94
:1014600000BF00BF00BF00BF207800F0010070BDCA
:1014700000C009202DE9F047744E80464FF0807778
:1014800030683C01724DB84249D100BF00BF00BF77
:1014900000BF00BF00BF00BF00BF00BF00BF00BF54
:1014A00000BF00BF00BF00BF00BF00BF00BF00BF44
:1014B00000BF00BF00BF00BF00BF00BF00BF00BF34
:1014C00000BF00BF00BF00BF00BFEC63152000F0ED
:1014D0006BFD002000F068FD00F0FF09AC6300BF69
:1014E00000BF00BF00BF00BF00BF00BF00BF00BF04
:1014F00000BF00BF00BF00BF00BF00BF00BF00BFF4
:1015000000BF00BF00BF00BF00BF00BF00BF00BFE3
:1015100000BF00BF00BF00BF00BF00BF00BF00BFD3
:1015200000BF00BF00BF00BF00BF00BF00BF00BFC3
:1015300000BF00BF00BF00BF00BF00BF00BF00BFB3
:1015400000BF00BF00BF00BF00BF00BF00BF00BFA3
:1015500000BF00BF00BF00BF00BF00BF00BFEC6303
:10156000062000F021FDAC6300BF00BF00BF00BF3C
:1015700000BF00BF00BF00BF00BF00BF00BF00BF73
:1015800000BF00BF00BF00BF00BF00BF00BF00BF63
:1015900000BF00BF00BF00BF00BF00BF00BF00BF53
:1015A00000BF00BF00BF00BF00BF00BF00BF00BF43
:1015B00000BF00BF00BF00BF00BF00BF00BF00BF33
:1015C00000BF00BF00BF00BF00BF00BF00BF00BF23
:1015D00000BF00BF00BF00BF00BF00BF00BF00BF13
:1015E00000BF00BF00BF00BFEC63012000F0DCFCC7
:1015F0004FEA880000F0D8FC3068B84202D1484673
:1016000000F0D2FCAC6300BF00BF00BF00BF00BF52
:1016100000BF00BF00BF00BF00BF00BF00BF00BFD2
:1016200000BF00BF00BF00BF00BF00BF00BF00BFC2
:1016300000BF00BF00BF00BF00BF00BF00BF00BFB2
:1016400000BF00BF00BFBDE8F087000054C1072005
:1016500000C009202DE9F041084C0F460646A56858
:1016600006E0A068401BB04202D30120BDE8F08133
:101670003846FFF7ABFE0028F3D1F7E7000009403A
:101680002DE9F04F89B0DFF8F0805FEA020B4FF0F0
:10169000000607910FD04FF4805501462A46684650
:1016A000FEF748FDDDE90047284603F047FE5FEA04
:1016B00000090DD017E086213048C8F80010092134
:1016C000016079462E480160862009B0BDE8F08FA0
:1016D00082212A48C8F80010222101607946284852
:1016E00001608220F1E7ABEB0605C7F580504FF0B3
:1016F000000AA84200D20546B5F5805F04D0204616
:10170000494600F0ADFFD8B907982A46811907EB82
:101710000900FEF719FD204600F0C2FD80B9204601
:10172000494600F00DF958B920464946FFF7C6FC76
:1017300078B10AF1010000F0FF0ABAF1030F05D3F6
:10174000484603F027FBD8F80000BEE7BAF1000FC7
:10175000E1D12E440027641C5E45C4D3484603F003
:1017600019FB06490020C8F80000086079460448C3
:1017700001600020A9E700006CC0072070C00720AE
:1017800074C007202DE9FF4F8DB00D46DDF868903D
:101790000026684C07935FEA09013ED04FF480575A
:1017A00001463A466846FEF7C5FCDDE900B10C91FA
:1017B0003A46691C6846FEF7BDFCDDE90010CDE93C
:1017C00004013A4668460F99FEF7B4FCDDE900854E
:1017D000A9EB0607C5F58050B84200D2074625B1EF
:1017E000D8457DD10C9885427AD14FF4805003F0D2
:1017F000A5FD5FEA000A1CD0D84550D10C9885425F
:101800004DD12A464FEA0830514600F0A1FE0006AD
:1018100019D5504603F0BEFA7AE08620206046488B
:1018200009210160784645490860862011B0BDE86D
:10183000F08F8220206040482221016079463F4895
:1018400001608220F2E70598804509D1049901EBF7
:101850000030C1F58052514400F07AFE0006D8D421
:10186000404600F01DFD0006D3D407983A46811982
:1018700005EB0A00FEF768FCEA194FEA083051460A
:1018800001F0A4FD0006C4D40599884533D104981D
:1018900000EB01300499C1F58052514427E00599CD
:1018A00088450AD1049800EB01300499C1F58052B3
:1018B000514600F04DFE0006ABD4404600F0F0FC6F
:1018C0000006A6D407983A4681190F98304401F0D3
:1018D0007DFD00069DD4059988450CD1049800E053
:1018E0000DE000EB01300499C1F58052514601F042
:1018F0006DFD00068DD4504603F04CFA0AE00798BF
:101900003A4681190F98304401F060FD000601D578
:1019100020688BE73E44002508F101084E45FFF49E
:1019200057AF0549002020600860784603490860E9
:1019300000207BE76CC0072070C0072074C0072020
:101940002DE9F34F0024484D484E494FC3B080461F
:101950004FF0820A4FF0210BA14641A94548FFF7FD
:1019600079FE00286CD101F003F902208DF8000007
:101970004FEA18108DF8010004EB08108DF80200F2
:1019800044988DF8039000EB04214FF4807201A875
:10199000FEF7DAFB00BF00BF00BF00BF00BF00BF03
:1019A00000BF00BF00BF00BF00BF00BF00BF00BF3F
:1019B00000BF00BF00BF00BF00BF00BF00BF00BF2F
:1019C00000BF00BF00BF00BF00BF00BF00BF00BF1F
:1019D00000BF00BF28494FF08050C8634FF48271A8
:1019E000684600F0EBFA24494FF08050886300BF4E
:1019F00000BF00BF00BF00BF00BF00BF00BF00BFEF
:101A000000BF00BF00BF00BF00BF00BF00BF00BFDE
:101A100000BF00BF00BF00BF00BF00BF00BF00BFCE
:101A200000BF00BF00BF00BF00BF00BF00BF641CFD
:101A3000E4B2102C91D341A90E48FFF70BFE48B138
:101A4000C5F800A07846C6F800B03860822045B0DE
:101A5000BDE8F08F01F040F8C5F800907846C6F870
:101A6000009038600020F2E76CC0072070C00720AB
:101A700074C00720A086010000C00920C906090E15
:101A8000002806DA00F00F0000F1E02080F8141DB5
:101A9000704700F1E02080F8001470472DE9F04312
:101AA000FE4800218162416821F440514160416C4F
:101AB00021F4405141F400514164F9494FF480024E
:101AC000CA610A6842F480020A60026822F4403265
:101AD0000260026C42F44032026487158F610A682A
:101AE00042F480720A60026922F440120261026DBF
:101AF00022F4401202650215CA650B6C23F4806360
:101B00000B64036923F440030361036D23F4400372
:101B100003654FF40069C1F85C900B6C23F400631B
:101B20000B64436823F4402343F480234360436CF5
:101B300023F4402343F400234364C36843F4403355
:101B4000C360C36C43F44033C364C36843F440438D
:101B5000C360C36C43F44043C364C36843F440733D
:101B6000C360C36C43F44073C364C36823F0407321
:101B7000C360C36C23F04073C36493048B630B6A2C
:101B800043F080530B62C36823F44063C360C36CAB
:101B900023F44063C364D3028B630C6A44F40014DF
:101BA0000C62446824F0406444F080644460446CF7
:101BB00024F0406444F000644464446824F04054D9
:101BC00044F080544460446C24F0405444F0005489
:101BD0004464C46824F0405444F00054C460C46CAD
:101BE00044F04054C464C46924F44024C461C46D06
:101BF00044F44024C465D403CC670C6E44F00074F4
:101C00000C66C46844F44054C460C46C24F440546A
:101C100044F40054C464446824F440644460446C54
:101C200024F440644464CB610B6823F400130B601C
:101C3000436823F003034360436C23F003039B1CBE
:101C4000436493018B610C6844F480340C604468F5
:101C500024F030044460446C24F0300444F0200448
:101C6000446414028C610D6845F480250D6005689C
:101C700025F040450560056C25F0404545F00045E0
:101C8000056455018D610E6846F400460E600669D4
:101C900026F440760661066D26F4407646F400761A
:101CA00006654FF0100CC1F858C00E6C46F01006D7
:101CB0000E64066926F0C0060661066D26F0C006B1
:101CC00046F08006066508268E65D1F8408048F00B
:101CD0000808C1F84080D0F8088028F04048C0F8D3
:101CE0000880D0F8488028F04048C0F848808D63CC
:101CF000D1F8208048F40048C1F82080D0F808804E
:101D000028F04058C0F80880D0F8488028F04058A3
:101D1000C0F848804FF48048C1F83880D1F820805E
:101D200048F48048C1F82080D0F8088028F4401892
:101D3000C0F80880D0F8488028F44018C0F84880DF
:101D40008A63D1F8208048F48068C1F82080D0F8F8
:101D5000088028F44028C0F80880D0F8488028F48B
:101D60004028C0F848804FF40078C1F83880D1F896
:101D7000208048F40078C1F82080D0F8088028F44A
:101D80004038C0F80880D0F8488028F44038C0F8BF
:101D900048808F630F6A47F480770F62876827F463
:101DA00040778760876C27F440778764C1F838C034
:101DB0000F6A47F010070F62876827F00C078760EB
:101DC000876C27F00C07876402278F630F6A47F040
:101DD00002070F62876827F003078760876C27F088
:101DE0000307876401278F630F6A47F001070F62BB
:101DF000076827F440170760076C27F4401707644B
:101E0000CA610A6842F480620A60026822F44002F1
:101E10000260026C22F440020264C1F81C900A685D
:101E200042F400620A60026822F040420260026CE2
:101E300022F040420264CD610A6842F400420A6026
:101E4000426822F003024260426C22F003024264C4
:101E5000CB610A6842F480320A60426822F00C02C8
:101E60004260426C22F00C0242645A00CA610D6862
:101E700045F400350D60456825F030054560456C3A
:101E800025F030054564CC610D6845F480250D6072
:101E9000056925F030050561056D03E000C00240CD
:101EA00000C0092025F0300505650425CD650D6CC1
:101EB00045F004050D64056925F0C0050561056D53
:101EC00025F0C0050565CE650D6C45F008050D646F
:101ED000C56825F00305C560C56C25F00305C5641C
:101EE000CB630B6A23F480330B62C36823F00C03CB
:101EF000C360C36C23F00C03C364CA630A6A22F490
:101F000000320A62C26822F03002C260C26C22F063
:101F10003002C264CC63086A20F480200862BDE805
:101F2000F083000010B5FEF771FBFEF79DFB04493E
:101F30004FF40052C1E90020A0F5F420886010BDE4
:101F4000B0C0072006493022C1F80822C1F81002AB
:101F5000D1F800028006FBD5D1F8140270470000CA
:101F600000C00050094804210161072101600021DF
:101F70004161416202214160C168C906FCD400E0B0
:101F80008168C1684907FBD4002070470080084081
:101F900000B50B46024604E0002000F005F802F808
:101FA000010B5B1EF8D200BD03498860C868C006FB
:101FB000FCD48868704700000080084000B50B46DC
:101FC000024603E012F8010BFFF7EEFF5B1EF9D2A9
:101FD00000BD00002DE9F84F6946384800F05AFC72
:101FE0008227374C374D384E4FF0220A002855D102
:101FF0009DF80000800701D400F0BAFD00BF00BFCB
:1020000000BF00BF00BF00BF00BF00BF00BF00BFD8
:1020100000BF00BF00BF00BF00BF00BF00BF00BFC8
:1020200000BF00BF00BF00BF00BF00BF00BF00BFB8
:1020300000BF00BF00BF00BF00BF00BFDFF88C9033
:102040004FF08058C9F83C806020FFF7ADFFC9F819
:10205000388000BF00BF00BF00BF00BF00BF00BF8F
:1020600000BF00BF00BF00BF00BF00BF00BF00BF78
:1020700000BF00BF00BF00BF00BF00BF00BF00BF68
:1020800000BF00BF00BF00BF00BF00BF00BF00BF58
:1020900000BF69460E4800F0FDFB38B12760784666
:1020A000C5F800A030608220BDE8F88F00202060D5
:1020B0002860784630600020F6E70000A086010026
:1020C0006CC0072070C0072074C0072000C0092022
:1020D00020A107002DE9F0474FF0000900BF00BF25
:1020E00000BF00BF00BF00BF00BF00BF00BF00BFF8
:1020F00000BF00BF00BF00BF00BF00BF00BF00BFE8
:1021000000BF00BF00BF00BF00BF00BF00BF00BFD7
:1021100000BF00BF00BF00BF00BF00BF314E4FF087
:102120008055F5639F20FFF73FFF0020FFF73CFF3E
:1021300000F0FF080020FFF737FFC4B20020FFF7D0
:1021400033FFC1B2B56300BF00BF00BF00BF00BF17
:1021500000BF00BF00BF00BF00BF00BF00BF00BF87
:1021600000BF00BF00BF00BF00BF00BF00BF00BF77
:1021700000BF00BF00BF00BF00BF00BF00BF00BF67
:1021800000BF00BF00BF184D184E194FB8F1BF0F68
:1021900003D1252C0AD0262C08D0822028602120AB
:1021A0003060784638608220BDE8F08711484129C8
:1021B00012D04FF48002422912D04A2910D0C0F820
:1021C0000090002000F0D0FAC5F800907846C6F8DC
:1021D000009038600020E7E74FF400110160F0E75D
:1021E0000260EEE700C009206CC0072070C0072025
:1021F00074C0072058C107202DE9F04FDFF8948004
:10220000DFF894B089B00F0004464FF0000628D0E4
:102210004FF4805501462A466846FDF78BFFDDE9FD
:1022200000A105912A46214606A8FDF783FFDDE9B6
:1022300006404FF00009BD1BC0F58051A94200D2F5
:102240000D4620B1544517D10599884214D1204636
:1022500000F026F800060FD5D8F8000009B0BDE858
:10226000F08F8621C8F800100921CBF800107946BC
:102270000A4801608620F1E72E44641C4846BE42AD
:10228000D9D3C8F800007946CBF8000003480160B4
:102290000020E3E76CC0072070C0072074C007204F
:1022A0002DE9FC47044601A93B4800F0F3FA3B4DF9
:1022B0003B4EDFF8F09048B182202860222079461A
:1022C00030608220C9F80010BDE8FC879DF804004A
:1022D000800701D400F04CFC20208DF8000020097C
:1022E0008DF8010020018DF8020000248DF80340D4
:1022F00000BF00BF00BF00BF00BF00BF00BF00BFE6
:1023000000BF00BF00BF00BF00BF00BF00BF00BFD5
:1023100000BF00BF00BF00BF00BF00BF00BF00BFC5
:1023200000BF00BF00BF00BF00BF00BF00BF00BFB5
:10233000DFF874804FF08057C8F83C70042168467D
:10234000FFF73CFEC8F8387000BF00BF00BF00BFF9
:1023500000BF00BF00BF00BF00BF00BF00BF00BF85
:1023600000BF00BF00BF00BF00BF00BF00BF00BF75
:1023700000BF00BF00BF00BF00BF00BF00BF00BF65
:1023800000BF00BF00BF00BF2C6079463460002052
:10239000C9F8001098E70000A08601006CC0072073
:1023A00070C0072074C0072000C009204FF480507F
:1023B00070470000014800687047000058C10720BE
:1023C00070B5044600BF00BF00BF00BF00BF00BF24
:1023D00000BF00BF00BF00BF00BF00BF00BF00BF05
:1023E00000BF00BF00BF00BF00BF00BF00BF00BFF5
:1023F00000BF00BF00BF00BF00BF00BF00BF00BFE5
:1024000000BF00BF174E4FF08055F5630520FFF762
:10241000CBFD0020FFF7C8FD2070B56300BF00BFF3
:1024200000BF00BF00BF00BF00BF00BF00BF00BFB4
:1024300000BF00BF00BF00BF00BF00BF00BF00BFA4
:1024400000BF00BF00BF00BF00BF00BF00BF00BF94
:1024500000BF00BF00BF00BF00BF00BF207800F07A
:10246000010070BD00C0092070B5044600BF00BF68
:1024700000BF00BF00BF00BF00BF00BF00BF00BF64
:1024800000BF00BF00BF00BF00BF00BF00BF00BF54
:1024900000BF00BF00BF00BF00BF00BF00BF00BF44
:1024A00000BF00BF00BF00BF00BF00BF174E4FF00E
:1024B0008055F5630520FFF777FD0020FFF774FDD9
:1024C0002070B56300BF00BF00BF00BF00BF00BFEA
:1024D00000BF00BF00BF00BF00BF00BF00BF00BF04
:1024E00000BF00BF00BF00BF00BF00BF00BF00BFF4
:1024F00000BF00BF00BF00BF00BF00BF00BF00BFE4
:1025000000BF00BF207800F0010070BD00C00920AE
:1025100070B50C4D0C4E0D4C2AB100F019F80006A8
:1025200009D5206870BD8620206009202860784683
:102530003060862070BD00202060286078463060C2
:10254000002070BD70C0072074C007206CC0072039
:102550002DE9FC5F3D4D3E4E3E4F5FEA020A8B4641
:1025600004464FF000080DD001A93B4800F092F955
:1025700080B1822028602120306078463860822037
:10258000BDE8FC9FC5F800807846C6F8008038603A
:102590000020F5E703208DF80000200C8DF80100E5
:1025A000200A8DF802008DF8034000BF00BF00BF75
:1025B00000BF00BF00BF00BF00BF00BF00BF00BF23
:1025C00000BF00BF00BF00BF00BF00BF00BF00BF13
:1025D00000BF00BF00BF00BF00BF00BF00BF00BF03
:1025E00000BF00BF00BF00BF00BF1C4C4FF08059B0
:1025F000C4F83C9004216846FFF7E0FC5146584679
:10260000FFF7C6FCC4F8389000BF00BF00BF00BF92
:1026100000BF00BF00BF00BF00BF00BF00BF00BFC2
:1026200000BF00BF00BF00BF00BF00BF00BF00BFB2
:1026300000BF00BF00BF00BF00BF00BF00BF00BFA2
:1026400000BF00BF00BF00BF9CE700006CC00720B8
:1026500070C0072074C00720A086010000C00920B8
:102660002DE9FC478A46044601A93A4800F012F9D0
:10267000394D3A4EDFF8E89048B182202860222098
:10268000794630608220C9F80010BDE8FC8703203D
:102690008DF8000020098DF8010020018DF802005E
:1026A00000248DF8034000BF00BF00BF00BF00BF83
:1026B00000BF00BF00BF00BF00BF00BF00BF00BF22
:1026C00000BF00BF00BF00BF00BF00BF00BF00BF12
:1026D00000BF00BF00BF00BF00BF00BF00BF00BF02
:1026E00000BF00BF00BFDFF87C804FF08057C8F804
:1026F0003C7004216846FFF761FC39145046FFF72F
:1027000047FCC8F8387000BF00BF00BF00BF00BF63
:1027100000BF00BF00BF00BF00BF00BF00BF00BFC1
:1027200000BF00BF00BF00BF00BF00BF00BF00BFB1
:1027300000BF00BF00BF00BF00BF00BF00BF00BFA1
:1027400000BF00BF00BF2C60794634600020C9F88C
:1027500000109AE7A08601006CC0072070C0072017
:1027600074C0072000C0092070B5064600BF00BF36
:1027700000BF00BF00BF00BF00BF00BF00BF00BF61
:1027800000BF00BF00BF00BF00BF00BF00BF00BF51
:1027900000BF00BF00BF00BF00BF00BF00BF00BF41
:1027A00000BF00BF00BF00BF00BF00BF384D4FF0EB
:1027B0008054EC635020FFF7F7FBAC6300BF00BF11
:1027C00000BF00BF00BF00BF00BF00BF00BF00BF11
:1027D00000BF00BF00BF00BF00BF00BF00BF00BF01
:1027E00000BF00BF00BF00BF00BF00BF00BF00BFF1
:1027F00000BF00BF00BF00BF00BF00BF00BF00BFE1
:1028000000BF00BF00BF00BF00BF00BF00BF00BFD0
:1028100000BF00BF00BF00BF00BF00BF00BF00BFC0
:1028200000BF00BF00BF00BF00BF00BF00BF00BFB0
:1028300000BF00BF00BF00BF00BF00BFEC630120AE
:10284000FFF7B2FBB000FFF7AFFBAC6300BF00BF08
:1028500000BF00BF00BF00BF00BF00BF00BF00BF80
:1028600000BF00BF00BF00BF00BF00BF00BF00BF70
:1028700000BF00BF00BF00BF00BF00BF00BF00BF60
:1028800000BF00BF00BF00BF00BF00BF70BD0000A1
:1028900000C009202DE9F041084C0F460646A56806
:1028A00006E0A068401BB04202D30120BDE8F081E1
:1028B0003846FFF785FD0028F3D1F7E7000009400F
:1028C0002DE9F041084C0F460646A56806E0A068D1
:1028D000401BB04202D30120BDE8F0813846FFF72B
:1028E000C3FD0028F3D1F7E7000009402DE9F04FC0
:1028F00089B0DFF8D080DFF8D0B05FEA02094FF08E
:10290000000607910FD04FF4805501462A466846CD
:10291000FDF710FCDDE90047284602F00FFD5FEAF5
:10292000000A0DD017E08621C8F800100921CBF865
:102930000010794625480160862009B0BDE8F08F77
:102940008221C8F800102221CBF8001079461F48D8
:1029500001608220F1E7A9EB0605C7F58050A84287
:1029600000D20546B5F5805F04D020465146FFF7FA
:1029700077FE80B92046FFF793FC60B907982A4696
:10298000811907EB0A00FDF7DFFB2E442046514674
:1029900000F044FA28B1504602F0FCF9D8F80000E3
:1029A000CBE70027641C4E45D5D3504602F0F2F920
:1029B0000020C8F800007946CBF800000348016009
:1029C0000020BAE76CC0072070C0072074C0072041
:1029D0002DE9FE430F46044602A93A48FFF75AFF85
:1029E000394D3A4EDFF8E88048B182202860222035
:1029F000794630608220C8F80010BDE8FE839DF85B
:102A00000800800701D400F0B3F802208DF8000020
:102A1000200C8DF80100200A8DF802008DF803408B
:102A20008DF8047000BF00BF00BF00BF00BF00BF33
:102A300000BF00BF00BF00BF00BF00BF00BF00BF9E
:102A400000BF00BF00BF00BF00BF00BF00BF00BF8E
:102A500000BF00BF00BF00BF00BF00BF00BF00BF7E
:102A600000BF00BF1B4F4FF08054FC630521684638
:102A7000FFF7A4FABC6300BF00BF00BF00BF00BFE8
:102A800000BF00BF00BF00BF00BF00BF00BF00BF4E
:102A900000BF00BF00BF00BF00BF00BF00BF00BF3E
:102AA00000BF00BF00BF00BF00BF00BF00BF00BF2E
:102AB00000BF00BF00BF0020286079463060C8F822
:102AC00000109AE7A08601006CC0072070C00720A4
:102AD00074C0072000C0092070B500BF00BF00BF50
:102AE00000BF00BF00BF00BF00BF00BF00BF00BFEE
:102AF00000BF00BF00BF00BF00BF00BF00BF00BFDE
:102B000000BF00BF00BF00BF00BF00BF00BF00BFCD
:102B100000BF00BF00BF00BF00BF144C4FF0805586
:102B2000E5630420FFF740FAA56300BF00BF00BFC4
:102B300000BF00BF00BF00BF00BF00BF00BF00BF9D
:102B400000BF00BF00BF00BF00BF00BF00BF00BF8D
:102B500000BF00BF00BF00BF00BF00BF00BF00BF7D
:102B600000BF00BF00BF00BF00BF70BD00C0092094
:102B700070B500BF00BF00BF00BF00BF00BF00BFF7
:102B800000BF00BF00BF00BF00BF00BF00BF00BF4D
:102B900000BF00BF00BF00BF00BF00BF00BF00BF3D
:102BA00000BF00BF00BF00BF00BF00BF00BF00BF2D
:102BB00000BF144C4FF08055E5630620FFF7F4F991
:102BC000A56300BF00BF00BF00BF00BF00BF00BFC4
:102BD00000BF00BF00BF00BF00BF00BF00BF00BFFD
:102BE00000BF00BF00BF00BF00BF00BF00BF00BFED
:102BF00000BF00BF00BF00BF00BF00BF00BF00BFDD
:102C000000BF70BD00C009202DE9F05F114EDFF854
:102C10004890DFF848A0150083460F464FF00008A3
:102C20000ED000240AE0395D0BEB0400FFF7D0FE64
:102C3000000602D53068BDE8F09F641CAC42F2D3B8
:102C4000C6F800807946C9F800800020CAF8001054
:102C5000F1E700006CC0072070C0072074C0072097
:102C60002DE9FF4F8DB00D46DDF868900026684CC9
:102C700007935FEA09013ED04FF4805701463A4678
:102C80006846FDF757FADDE900B10C913A46691C38
:102C90006846FDF74FFADDE90010CDE904013A4638
:102CA00068460F99FDF746FADDE90085A9EB0607AE
:102CB000C5F58050B84200D2074625B1D8457DD130
:102CC0000C9885427AD14FF4805002F037FB5FEACE
:102CD000000A1CD0D84550D10C9885424DD12A46C7
:102CE0004FEA08305146FFF733FC000619D550462D
:102CF00002F050F87AE08620206046480921016001
:102D0000784645490860862011B0BDE8F08F8220E2
:102D1000206040482221016079463F4801608220BE
:102D2000F2E70598804509D1049901EB0030C1F51F
:102D300080525144FFF70CFC0006D8D44046FFF700
:102D4000AFFA0006D3D407983A46811905EB0A007A
:102D5000FDF7FAF9EA194FEA08305146FFF754FF38
:102D60000006C4D40599884533D1049800EB01309E
:102D70000499C1F58052514427E0059988450AD14C
:102D8000049800EB01300499C1F580525146FFF7D9
:102D9000DFFB0006ABD44046FFF782FA0006A6D45C
:102DA00007983A4681190F983044FFF72DFF000627
:102DB0009DD4059988450CD1049800E00DE000EB06
:102DC00001300499C1F580525146FFF71DFF0006FE
:102DD0008DD4504601F0DEFF0AE007983A4681198B
:102DE0000F983044FFF710FF000601D520688BE7ED
:102DF0003E44002508F101084E45FFF457AF054950
:102E000000202060086078460349086000207BE7C6
:102E10006CC0072070C0072074C007202DE9F34F55
:102E200083B0044601A97148FFF734FD704D714E1F
:102E3000714F4FF0820818B12120C5F800806CE076
:102E40009DF80400800701D4FFF792FEAD208DF8B5
:102E5000000020098DF8010020018DF802004FF0DC
:102E6000000B8DF803B000BF00BF00BF00BF00BF64
:102E700000BF00BF00BF00BF00BF00BF00BF00BF5A
:102E800000BF00BF00BF00BF00BF00BF00BF00BF4A
:102E900000BF00BF00BF00BF00BF00BF00BF00BF3A
:102EA00000BF00BF00BFDFF854914FF0805A544676
:102EB000C9F83CA004216846FFF780F80221049875
:102EC000FFF77CF8C9F8384000BF00BF00BF00BF63
:102ED00000BF00BF00BF00BF00BF00BF00BF00BFFA
:102EE00000BF00BF00BF00BF00BF00BF00BF00BFEA
:102EF00000BF00BF00BF00BF00BF00BF00BF00BFDA
:102F000000BF00BF00BF00BF022401A93748FFF780
:102F1000C1FC48B12220C5F8008030607846386096
:102F2000822005B0BDE8F08F00BF00BF00BF00BF2A
:102F300000BF00BF00BF00BF00BF00BF00BF00BF99
:102F400000BF00BF00BF00BF00BF00BF00BF00BF89
:102F500000BF00BF00BF00BF00BF00BF00BF00BF79
:102F600000BF00BF00BF00BFC9F83CA0AD20FFF705
:102F70001BF8049802212044FFF720F8C9F838A074
:102F800000BF00BF00BF00BF00BF00BF00BF00BF49
:102F900000BF00BF00BF00BF00BF00BF00BF00BF39
:102FA00000BF00BF00BF00BF00BF00BF00BF00BF29
:102FB00000BF00BF00BF00BF00BF00BF00BF00BF19
:102FC000A41CA4B2B4F5805F9FD301A90748FFF702
:102FD00061FC00287FF430AFFFF77EFDC5F800B03C
:102FE0007846C6F800B0386000209AE7A086010055
:102FF0006CC0072070C0072074C0072000C00920E3
:103000004FF4805070474FF4800070472DE9F04F27
:1030100089B0DFF8D080DFF8D0B05FEA02094FF066
:10302000000607910FD04FF4805501462A466846A6
:10303000FDF780F8DDE90047284602F07FF95FEAF6
:10304000000A0DD017E08621C8F800100921CBF83E
:103050000010794625480160862009B0BDE8F08F50
:103060008221C8F800102221CBF8001079461F48B1
:1030700001608220F1E7A9EB0605C7F58050A84260
:1030800000D20546B5F5805F04D020465146FFF7D3
:10309000E7FA80B92046FFF703F960B907982A4696
:1030A000811907EB0A00FDF74FF82E4420465146E0
:1030B00000F096FA28B1504601F06CFED8F80000F6
:1030C000CBE70027641C4E45D5D3504601F062FE85
:1030D0000020C8F800007946CBF8000003480160E2
:1030E0000020BAE76CC0072070C0072074C007201A
:1030F0002DE9FF4703A93B48FFF7E2FB3A4D3B4E62
:10310000DFF8EC9050B182202860212079463060B1
:103110008220C9F8001004B0BDE8F0879DF80C00CB
:10312000800701D4FFF724FD42208DF80000002421
:10313000CDF80140CDF80540ADF8094000BF00BF13
:1031400000BF00BF00BF00BF00BF00BF00BF00BF87
:1031500000BF00BF00BF00BF00BF00BF00BF00BF77
:1031600000BF00BF00BF00BF00BF00BF00BF00BF67
:1031700000BF00BF00BF00BF00BF00BFDFF874800A
:103180004FF08057C8F83C700B216846FEF716FFD9
:10319000C8F8387000BF00BF00BF00BF00BF00BF4D
:1031A00000BF00BF00BF00BF00BF00BF00BF00BF27
:1031B00000BF00BF00BF00BF00BF00BF00BF00BF17
:1031C00000BF00BF00BF00BF00BF00BF00BF00BF07
:1031D00000BF00BF2C60794634600020C9F80010A1
:1031E00099E70000A08601006CC0072070C007208E
:1031F00074C0072000C009202DE9F34F85B00446B4
:1032000003A96D48FFF75CFB6C4D6D4E6D4F4FF0A1
:10321000820B18B12120C5F800B060E0FFF7A8FCD0
:1032200042208DF800004FF0000ACDF801A0CDF843
:1032300005A0ADF809A000BF00BF00BF00BF00BFE0
:1032400000BF00BF00BF00BF00BF00BF00BF00BF86
:1032500000BF00BF00BF00BF00BF00BF00BF00BF76
:1032600000BF00BF00BF00BF00BF00BF00BF00BF66
:1032700000BF00BF00BFDFF850914FF08058C9F881
:103280003C800B216846FEF799FEC9F8388000BFE4
:1032900000BF00BF00BF00BF00BF00BF00BF00BF36
:1032A00000BF00BF00BF00BF00BF00BF00BF00BF26
:1032B00000BF00BF00BF00BF00BF00BF00BF00BF16
:1032C00000BF00BF00BF00BF00BF00BF00BF03A919
:1032D0003948FFF7F5FA48B12220C5F800B0306050
:1032E00078463860822007B0BDE8F08F9DF80C006A
:1032F000800701D4FFF73CFC02208DF80000200C71
:103300008DF80100200A8DF8020006988DF8034020
:103310008DF8040000BF00BF00BF00BF00BF00BFAA
:1033200000BF00BF00BF00BF00BF00BF00BF00BFA5
:1033300000BF00BF00BF00BF00BF00BF00BF00BF95
:1033400000BF00BF00BF00BF00BF00BF00BF00BF85
:1033500000BF00BF4446C846C9F83C400521684646
:10336000FEF72CFEC8F8384000BF00BF00BF00BF0A
:1033700000BF00BF00BF00BF00BF00BF00BF00BF55
:1033800000BF00BF00BF00BF00BF00BF00BF00BF45
:1033900000BF00BF00BF00BF00BF00BF00BF00BF35
:1033A00000BF00BF00BF00BFC5F800A07846C6F848
:1033B00000A03860002096E7A08601006CC00720BE
:1033C00070C0072074C0072000C009202DE9F05FFD
:1033D000114EDFF84890DFF848A0150083460F46ED
:1033E0004FF000080ED000240AE0395D0BEB04001A
:1033F000FFF702FF000602D53068BDE8F09F641CAD
:10340000AC42F2D3C6F800807946C9F800800020AB
:10341000CAF80010F1E700006CC0072070C0072058
:1034200074C007202DE9FF4F8DB00D46DDF8689080
:103430000026684C07935FEA09013ED04FF480579D
:1034400001463A466846FCF775FEDDE900B10C918D
:103450003A46691C6846FCF76DFEDDE90010CDE9CF
:1034600004013A4668460F99FCF764FEDDE90085E1
:10347000A9EB0607C5F58050B84200D2074625B132
:10348000D8457DD10C9885427AD14FF4805001F017
:1034900055FF5FEA000A1CD0D84550D10C988542F0
:1034A0004DD12A464FEA08305146FFF751F8000641
:1034B00019D5504601F06EFC7AE08620206046481F
:1034C00009210160784645490860862011B0BDE8B1
:1034D000F08F8220206040482221016079463F48D9
:1034E00001608220F2E70598804509D1049901EB3B
:1034F0000030C1F580525144FFF72AF80006D8D4B5
:103500004046FEF7CDFE0006D3D407983A4681190F
:1035100005EB0A00FCF718FEEA194FEA083051469D
:10352000FFF754FF0006C4D40599884533D10498A9
:1035300000EB01300499C1F58052514427E0059910
:1035400088450AD1049800EB01300499C1F58052F6
:103550005146FEF7FDFF0006ABD44046FEF7A0FE45
:103560000006A6D407983A4681190F983044FFF711
:103570002DFF00069DD4059988450CD1049800E0E4
:103580000DE000EB01300499C1F580525146FFF780
:103590001DFF00068DD4504601F0FCFB0AE00798A1
:1035A0003A4681190F983044FFF710FF000601D505
:1035B00020688BE73E44002508F101084E45FFF4E2
:1035C00057AF05490020206008607846034908602D
:1035D00000207BE76CC0072070C0072074C0072064
:1035E0002DE9F34F00244A4D4A4E4B4FC3B080465D
:1035F0004FF0820A4FF0210BA14641A94748FFF73F
:103600005FF9002870D19DF80401800701D4FFF70D
:10361000AFFA02208DF800004FEA18108DF8010073
:1036200004EB08108DF8020044988DF8039000EB2D
:1036300004214FF4807201A8FCF786FD00BF00BF93
:1036400000BF00BF00BF00BF00BF00BF00BF00BF82
:1036500000BF00BF00BF00BF00BF00BF00BF00BF72
:1036600000BF00BF00BF00BF00BF00BF00BF00BF62
:1036700000BF00BF00BF00BF00BF00BF28494FF020
:103680008050C8634FF482716846FEF797FC244966
:103690004FF08050886300BF00BF00BF00BF00BF75
:1036A00000BF00BF00BF00BF00BF00BF00BF00BF22
:1036B00000BF00BF00BF00BF00BF00BF00BF00BF12
:1036C00000BF00BF00BF00BF00BF00BF00BF00BF02
:1036D00000BF00BF00BF641CE4B2102C8DD341A911
:1036E0000E48FFF7EDF848B1C5F800A07846C6F8D7
:1036F00000B03860822045B0BDE8F08FFFF7ECF9EC
:10370000C5F800907846C6F8009038600020F2E7CF
:103710006CC0072070C0072074C00720A08601007D
:1037200000C00920F8B51446074E0A460B19716807
:1037300000258B4200D90A1B034600943068FDF730
:10374000DBF82846F8BD0000B0C0072070B503467E
:1037500008468D180549002449688D4200D9881A09
:103760001946FDF793F8204670BD0000B0C0072051
:1037700010B5FCF744FEFCF79BFD07481922416891
:10378000491CB1FBF2F3416002FB1311002902D185
:103790000168491C016010BDF8C0072010B54FF04A
:1037A000E02440F2527060611F216017FEF766F955
:1037B0000020A0610720206110BD0000094810B55D
:1037C000022141600021016741610B22C260C16397
:1037D00001214160FFF7E2FF0221C81EFEF74EF90A
:1037E000002010BD000009404F4810B52021C0F84E
:1037F000A01100BFD0F8A0114906FBD50521C0F8E3
:1038000004114FF04472C0F8A8214FF48062C0F850
:10381000AC210122C0F80C210B23C0F88430C0F881
:103820008020AA22C0F88C205523C0F88C3000BF1D
:10383000D0F888406401FBD50324C0F88040C0F86C
:103840008C20C0F88C30C0F808113849C0F8C4107A
:103850000021C0F8C811D0F888106FEA11618A07FA
:103860003349D0F80C2102F0030207D07AB3012AC1
:1038700044D0022A47D0032A4ED13AE02AB1012A85
:1038800013D0022A24D0032A46D1D0F88820D0F8B9
:103890000431C2F30742DBB2521C5B1C5A43D0F81E
:1038A0008830244CC3F30E030EE0D0F88820D0F803
:1038B0000431C2F30742DBB2521C5B1C5A43D0F8FE
:1038C00088301D4CC3F30E035B1C634321E010E002
:1038D000D0F88820D0F80431C2F30742DBB2521C82
:1038E0005B1C5A43D0F888304FF47A44C3F30E037C
:1038F000EAE7D0F80421114BD2B209E0D0F8042154
:103900000F4BD2B204E0D0F804214FF4FA43D2B204
:10391000521CB3FBF2F20A60016821F4704141F4D9
:103920000051016010BD000000C00F40DE96EA8724
:1039300000C1072000127A0000366E0100093D0028
:10394000001BB70070B51C4B186818601B481C4A58
:103950001C490578DC01D5B1466800251EB14368D5
:103960005B1E436002E002265E609D600570D068C9
:1039700020F44050D060D06C20F4405040F400500F
:10398000D064CC63086A40F48000086270BD43686C
:1039900073B1D36823F44053D360D36C23F4405302
:1039A00043F40053D3648C630A6A42F480020A62CF
:1039B0000121017070BD0000008000404CC1072053
:1039C00000C0024000C0092000B5FCF711FD044909
:1039D0005DF804EB41EA0040891300F015BD0000DA
:1039E0000005400010B502468078FCF701FD0B4948
:1039F000D1F84432012484402343C1F84432C1F851
:103A000048029088C1F84C02D1F80002C005FBD5ED
:103A10004FF48070C1F8080210BD000000C00050D3
:103A200010B500B101204FF4807444EA004107480A
:103A300000F0EAFC06480321C0F84412D0F8001256
:103A4000C905FBD5C0F8084210BD00000005D8002C
:103A500000C000507047000010B5040001D00120E4
:103A600000E000204FF4807141EA0041054800F079
:103A7000CBFC05494FF000700CB1886710BDC867DA
:103A800010BD00000005FE0000C0092010B5084C64
:103A9000A288402A00D940228020216800F06AFCD8
:103AA000216801442160A188081AA08010BD00008F
:103AB000E0C0072010B5064C0020216800F034FA61
:103AC000216801442160A188081AA08010BD00006F
:103AD000E0C007207047000000B5FCF789FC0449EE
:103AE0005DF804EB41EA0040024900F08DBC0000A3
:103AF000000540000001200000B5FCF779FC0449F6
:103B00005DF804EB41EA0040891300F07DBC000041
:103B1000000540002DE9F0414A4C0027A4F10806B9
:103B20002178A4F11C05082864D2DFE800F06304C2
:103B300065746363868400F0FDFB2078C009FFF79D
:103B4000C9FFE088B0802078C0F34111F1BB6178F3
:103B50000C294BD2DFE801F006094A0B4A101B1E64
:103B60002026324300F0B6F84EE0002000E00120AD
:103B700000F068FA50B306E010F01F0F36D1A078BD
:103B800040F080002870BDE8F04100F0D9BB00F0A3
:103B900065F839E000202AE010F01F0F26D12948EF
:103BA0001B381AE010F01F0F20D100F093FA68B113
:103BB00000F0C6FBBDE8F041FFF74CBF00F01F006E
:103BC000012813D1687808B1207900E00EE0A978C7
:103BD00088420BD21B490C39084430601DE000F0CC
:103BE0001F00012802D100F01DFBC3E7802000F078
:103BF00091FBB780BDE8F081080608D4B0880028A2
:103C0000F8D0FFF757FFB0880028EFD0F2E7BDE803
:103C1000F04100F09BBB080603D5BDE8F041FFF77B
:103C200035BF28780106E5D500F07F002870BDE893
:103C3000F04100F0F3B9802000E00020BDE8F04141
:103C4000FFF7C2BEE8C00720022803D0032803D133
:103C5000FCF750BFFCF770BF70470000194810B563
:103C6000007810F01F0F1748C07829D1154908397E
:103C7000012806D0134A0228937806D003281FD1C2
:103C800012E011480860122012E01048002204E0FF
:103C900004780CB144882044521C9342F8D1027835
:103CA00072B10860408803E0094818440860007851
:103CB0008A88824200D98880FFF7E8FE012010BD83
:103CC000002010BDE8C00720F05B0000025C00008F
:103CD000235C000070B51D481C4D0078A5F1080557
:103CE00010F01F040AD01948A5F11401184B4A78A6
:103CF0000079012C06D0022C26D109E0134818388F
:103D000028601DE002B3897888421DD2002015E0AA
:103D100000F08F04200605D504F00F064FF4803024
:103D2000B04001E00120A0400AB922070CD18A6806
:103D3000024209D0C9680142E8D0012018802B60F6
:103D4000FFF7A4FE012070BD002070BDE8C0072071
:103D500064DD07202DE9F0412F4DD5F80032C5F87C
:103D60000832180721D52D4800F040FB2C48FEF7FB
:103D7000E9F8C10605D500F00DF9BDE8F04100F005
:103D800041B9810705D5BDE8F04100F0010000F020
:103D900079B8010709D5400703D5BDE8F04100F027
:103DA000DBBABDE8F04100F037B91E4E58074FF0BE
:103DB00001071DD4BDE8F0815FF00004D5F8302282
:103DC00007FA04F10A4210D06008C5F8381200BFA3
:103DD000D5F800128906FBD5D5F81412E2070CD0ED
:103DE00056F8201009B103208847641C202CE5D325
:103DF000D5F830020028DFD1DCE73CB9490705D50A
:103E0000316819B1012088470124D7E756F82010FE
:103E10000029EAD00220E7E700C000500005FE00BC
:103E20000002FE00945C0000134800B5C16821F058
:103E3000405141F00051C160C16C41F04051C1643A
:103E40000E491A200860091D0A6830EA0202FBD1F7
:103E50004FF0E0214FF08070C1F88002084B202223
:103E600083F80024C1F8000100F094F800205DF808
:103E700004EB00F0D3B8000000C00240F4CF0050C3
:103E800018E000E0002802D1014901204870704785
:103E9000F0C0072070B5194C607820B30026184D8B
:103EA000012810D002280DD1A8686168401A154970
:103EB000884207D31448406B400003D50120FFF728
:103EC000CBFD667070BDA8686168401A0F498842D2
:103ED000F8D30020FFF7C0FDA86860600220607082
:103EE00026700BA005E020780028EBD1012020707F
:103EF0000AA0BDE87040FCF7DDBD0000F0C007205F
:103F000000000940A086010000C0092040420F00C7
:103F10002055536220457272000000002020626F1D
:103F20006F7420200000000000F00F02012370B524
:103F300003EB8203154AC2F8283200BFD2F82032C0
:103F40001C05FBD5C3F309030024DD1C05E000BFFD
:103F5000D2F8186241F8046B641CB4EB950FF7D3E8
:103F60000021C2F8281241F24821C140C9070AD1F4
:103F7000FCF73EFA4FF4A06141EA004000F036FA47
:103F8000034800F033FA184670BD000000C000502E
:103F90000005F2000D480021C0F848124021C0F889
:103FA0004C120122C0F84822C0F84C12D0F800127E
:103FB000C905FBD54FF0FF31C0F83812C0F83412F4
:103FC000C0F808120C21C0F80412704700C000505D
:103FD000044800214FF00112818001704170C0E956
:103FE00002217047CCC0072000B5FCF701FA044954
:103FF0005DF804EB41EA0040891300F005BA0000C7
:104000000005400010B5FFF7E3FF024900204870AB
:1040100010BD0000F0C007207047000030B5074910
:10402000074D41EA00442146284600F0EDF92146BB
:104030002846BDE8304000F0E7B9000000018000EC
:104040000005D00070B502462148A0F11C0401789B
:1040500011F01F030146498804D0012B29D0022BFF
:1040600027D111E0012924D132B1012000F080F9DB
:10407000A08840F0020005E0002000F079F9A08857
:1040800020F00200A08021E0007900F08F000306FC
:1040900005D500F00F034FF480359D4001E0012568
:1040A000854063782BB1030703D0A3682B4200D06F
:1040B00009B1002070BD22B100F02CF9E06828435E
:1040C00003E0FFF781FCE068A843E060012070BDD9
:1040D000E8C007202DE9F84F504F00200090B87835
:1040E0004FF000094FF0010A4FF4803BA7F11C0686
:1040F00000286AD04A4C64E06078022804D0042882
:1041000040D005285BD140E06179B878814237D151
:1041100070702079B070414900200C3901F800908E
:10412000401C0428FAD301254FEA06080AFA05F0D4
:10413000D8F80810084202D02846FFF7CDFCD8F87E
:1041400008100BFA05F0084203D045F08000FFF795
:10415000C3FC6D1C102DE9D34FF00110C8E9020912
:104160000120FFF75DFCE0794006B8F8040002D5B5
:1041700040F0010001E020F00100A8F804001EE07A
:1041800060881DE0E078009019E00098B8B9A07848
:1041900000F08F05280604D505F00F010BFA01F099
:1041A00001E00AFA05F0B16801432046B160FFF76B
:1041B00019FC2846FFF7A0FC2846FFF715FF2078DA
:1041C00004442078002897D11FE086F8019001244C
:1041D0005546D846B16805FA04F0084202D0204698
:1041E000FFF77AFCB16808FA04F0084203D044F003
:1041F0008000FFF771FC641C102CEBD34FF0011012
:10420000C6E902090020FFF70BFCB87871788842F4
:1042100002D10120BDE8F88F0020FBE7E8C00720AD
:10422000025C00002DE9FC5F384D00273E466878AF
:10423000BB46B846002866D0BA46354C05F11C0985
:104240005DE06078022804D0042808D0052854D105
:1042500019E06079697888424FD060884EE0A7788D
:1042600099F80410E6784FF00008B94245D199F862
:104270000200B04241D125484FF0010A103010F839
:1042800007B0C65539E099F80410B94235D1A17884
:1042900001F08F010191090605D5019901F00F0286
:1042A0004FF4803101E0019A01219140009199F889
:1042B0000200B04213D1A8680843A860E9680098DA
:1042C00081432046E960FFF78DFB0198FFF714FC5E
:1042D0000198FFF789FE009948EA01080DE05E4564
:1042E0000BD118EA010F08D1A8688843A860E868D4
:1042F0008843E8600198FFF7EFFB207804442078BA
:1043000000289ED15046BDE8FC9F0000CCC007208D
:10431000025C000000B5FCF76BF804495DF804EBA3
:1043200041EA0040024900F06FB80000000540007B
:104330000001010001490020FFF7F6BDE8C0072099
:1043400000221146802000F015B80000014900202D
:10435000FFF7EABD64DD07200348012141700349EE
:104360008968416070470000F0C0072000000940E4
:104370007047000070B513460546134C00F00F005F
:10438000022202EB8000C4F82802C4F82432002084
:10439000DA1C04E051F8046BC4F81C62401CB0EB5A
:1043A000920FF7D30020C4F828022846FCF720F823
:1043B0004FF4A06141EA004000F018F8034800F013
:1043C00015F8184670BD000000C000500005FA0046
:1043D00004480168044A01F4E06111430160BFF33D
:1043E0004F8FFEE70CED00E00400FA0505491022AE
:1043F000C1F80822C1F81002D1F80002C006FBD5AE
:104400007047000000C00050094A1023C2F808326B
:10441000C2F81002D2F80002C006FBD5C2F808327A
:10442000C2F81012D2F80002C006FBD57047000097
:1044300000C000502A4A93782A4A012B04D003294D
:1044400002D809B1082803D9506980022BD544E06D
:1044500000EB40000844C0B219283ED2DFE800F06B
:104460003D0D0F11131517191B1D1F21232527297A
:104470002B2D2F31333537393B000D20704712205B
:1044800070471420704705207047062070470720AA
:1044900070470220704703207047042070471520A2
:1044A00070470F207047132070470820704709207D
:1044B00070470A207047102070471120704716205F
:1044C00070470E2070471720704718207047012052
:1044D00070470B2070470C20704700207047000089
:1044E00004C1072000C0092008494A6BD20301D447
:1044F000012202704A6B920301D402220270496BBE
:10450000490301D4032101700020704700C0092035
:104510002DE9F0470446FCF7B9FAA0F1C871624AE8
:1045200017394FF480354FF008034FF480284FF4CB
:1045300000407DD0012901D002297AD15B490E6863
:1045400026F440160E600E6C26F440160E644FF4EE
:104550008069C2F81C90166846F4806616600E6882
:1045600026F440060E600E6C26F440060E644FF4EE
:10457000006AC2F81CA0166846F4006616600E6851
:1045800026F040460E600E6C26F040460E64D06168
:10459000166846F4004616604E6826F003064E6024
:1045A0004E6C26F003064E64D561166846F48036DC
:1045B00016604E6826F00C064E604E6C26F00C0617
:1045C0004E644FF40036D661176847F40037176021
:1045D0004F6827F030074F604F6C27F030074F646B
:1045E000C2F81C80176847F4802717600F6927F00E
:1045F00030070F610F6D27F030070F650427D7656F
:10460000D2F840C04CF0040CC2F840C0D1F810C041
:104610002CF0C00CC1F810C0D1F850C02CF0C00C68
:10462000C1F850C0D365116C41F00801116401E07C
:104630001CE01AE0E10701D1C2F81890A10701D4EB
:10464000C2F818A0610700D49061200700D49561DA
:10465000E00600D49661A00601D4C2F81880600676
:1046600000D4976520061BD4936519E09561936586
:104670000021D061260602D5C2F81C8001E0C2F8F4
:1046800018806406240ED0619061491CC9B20829C3
:10469000EFD3D061D561D36595619365D561D3655D
:1046A0000020BDE8F087000000C0092000C00240E3
:1046B00010B5FCF7EBF94249082217384FF4803364
:1046C000B0F1C87077D0012801D0022875D13D48DB
:1046D000046824F440140460046C24F4401404645A
:1046E0000415CC610C6844F480640C60046824F404
:1046F00040040460046C24F440040464C414CC61D9
:104700000C6844F400640C60046824F040440460C5
:10471000046C24F0404404644FF40044CC610C6801
:1047200044F400440C60446824F003044460446C86
:1047300024F003044464CB610B6843F480330B60C2
:10474000436823F00C034360436C23F00C03436481
:104750004FF40033CB610B6843F400330B604368C4
:1047600023F030034360436C23F0300343644FF481
:104770008023CB610B6843F480230B60036923F033
:1047800030030361036D23F0300303650423CB651D
:104790000B6C43F004030B64036923F0C003036153
:1047A000036D23F0C0030365CA65086C40F0080080
:1047B000086402E0FFE78B618A65002010BD0000FD
:1047C00000C0092000C002402DE9F0431949012230
:1047D0008A6302238B6310248C634FF48079C1F8C1
:1047E00038900D158D6396028E6397038F634FF497
:1047F000004CC1F838C0082819D2DFE800F00407DF
:10480000090B0D101214C1F83CC00DE0CF630BE092
:10481000CE6309E0CD6307E0C1F83C9004E0CC63CF
:1048200002E0CB6300E0CA630020BDE8F0834FF0F4
:10483000FF30FAE700C0092002E008C8121F08C1D3
:10484000002AFAD170477047002001E001C1121F11
:10485000002AFBD170470000F0B505460020034652
:1048600002462B4C4FF4007700E05B1CEE5C46B137
:1048700002EB030CA4440CF5805C9CF800C8B44522
:10488000F3D0032B3FD302F5C0502044037F457F74
:10489000C67F03EB0523857F2D0405EB06652B44BE
:1048A00051EA03052BD021B91A49496840318B429E
:1048B00025D8194B00215518254405F5805595F844
:1048C00000585D54491C0C29F5D3817EC27E01EB52
:1048D0000221027D407D120402EB00600C1820468C
:1048E00000F062FD40F6F57502E000BF00F05CFDEF
:1048F000C11EA942FAD3A0F57061FF3901D0002092
:10490000F0BD2046F0BD2032BA42AFD3F0BD00006A
:1049100081C1072078C00720EDDB0720F8B50A4CDD
:1049200000210091A56800EB4001C1EBC01668466C
:1049300000F058FA30B1A068401BB0EBC60FF6D3B8
:104940000020F8BD0098F8BD000009408CB046205A
:104950008DF814004FF000098DF8179037208DF86E
:104960001500DFF830B332208DF81600DBF80000B8
:10497000CA464FF6FF031840C74B40F480701843F7
:10498000CBF80000C548C749C94DC0F800A0C448CD
:104990000068A0F56C50FF380860C34900F5E0508E
:1049A0000860C249400A0860F8202870FF2068703B
:1049B000A870FBF7A5FCC04CBE49002094F9052067
:1049C00051F822102A1802F580520B5C401C82F824
:1049D00000386028F6D34FF4E175294640F24910BB
:1049E000FBF768FC294640F29F10FBF763FCDFF8F9
:1049F000CC824FF40055207808B1FFF74BFAA0792C
:104A000028B101281AD0207800286FD00CE10A20A4
:104A1000FBF7F7FCAAA0FCF74DF8FBF723FD0028F5
:104A200079D10120A0714FF4005584F803A006202D
:104A3000FBF7E7FC0A20FBF7E4FC03E11922294617
:104A40009E48FCF74DF898F8180000287DD098F89B
:104A5000000006287ED2DFE800F07D030B4A4A4DB5
:104A600040F2044000880490D8F80410814271D0CC
:104A700098F809004FF00109474601286AD1D7F894
:104A80000A0018B991488069C7F80A0090A0FCF79D
:104A900011F80026B84617E00720FBF7B2FCD7F85C
:104AA0000E00B846871B402F00D94027A9193A4667
:104AB0008A481931FCF714F8D8F80A003A4630440D
:104AC000864900F0CDFD3E44D8F80E004746B0427E
:104AD000E2D8397801293DD10A064FF0E021C1F82A
:104AE0008021D7F80A0000F027F933E095E04FF075
:104AF000010932E098F809004FF001094746032800
:104B00002BD177A0FBF7D6FF6549784800260A68C5
:104B1000B846026017E07DE00720FBF772FCD7F88B
:104B20000E00871B402F00D94027A9193A466B4831
:104B30001931FBF7D5FF5A483A4600688119674892
:104B4000FEF7F0FD3E44474600E025E0D8F80E00B1
:104B5000B042E1D898F81800F0B198F8080046463D
:104B6000C00614D561494FF400500122086005F1D8
:104B7000180104A8CDF810A0FEF7E8FD307820B1A8
:104B8000C8214FF47A70FBF795FB307E20B1307A64
:104B9000800701D5FFF71CFCD8F80E001B35054433
:104BA0004648FBF77BFF50B30220A07150484FF4FA
:104BB000005580F800A00B20FBF723FCB9F1000F93
:104BC0001DD04C484FF00009826842F21073816892
:104BD000891A9942FBD34FF42F714FF47A70FBF787
:104BE00069FB45A0FBF766FF4648406D400502D5CE
:104BF00000200A9001E00A9808B9FFF7E9FBE07885
:104C0000401CC0B2E0700C2802D30120A07001E06B
:104C1000A078B8B1FBF7E0FE14E001202070FFF7A8
:104C200003F90120FEF718FF3148007850B1002148
:104C300005A8FFF711FE28B184F806A04FF400552F
:104C400084F803A009A800F0CDF89DF824001928E5
:104C50007FF4D1AE2C48416821F440514160416C51
:104C600021F4405141F40051416426484FF4800141
:104C7000C161016841F480010160DBF80010064A5F
:104C800001F4E061121D1143CBF80010BFF34F8F08
:104C9000FEE700000CED00E00000FA05ACC00720C4
:104CA000B8C007209CC0072094C0072098C00720E8
:104CB00081C1072060C00720BCC0072068C1072051
:104CC0002020636865636B2000000000005B00002B
:104CD000464C41534820312000000000F9DB0720FA
:104CE000464C41534820322000000000B0C007204D
:104CF00068C0072000000940204C4F4164456420F3
:104D00000000000000C0092000C00240084A34230F
:104D10001360C2E9010107484FF47A710068B0FBE3
:104D2000F1F0D06002F11401104600F03FBA00002B
:104D30003CDC072000C1072072B60349034A01404A
:104D40001160FBF7CDB9000080FFFF1F08ED00E008
:104D500010B572B606240E4951F82420824212D9A9
:104D60000B49783951F82410814207D12146084671
:104D700000F042FB21460846FFF7C8FF21460846DF
:104D800000F03AFB02E0641C1D2CE5D962B610BDB0
:104D9000785B000010B5002821D0114B0022001FC5
:104DA000196803E0814203D80A4649680029F9D10D
:104DB00052B11368841A9C4204D1006818441060F0
:104DC000104602E0506000E0186039B102680B1A2A
:104DD000934203D10B681A4402604968416010BDD8
:104DE00060C1072006490A78012A02D04FF0FF303F
:104DF000704700220A70C9780170104670470000A1
:104E000004C10720F8B56E4C00258DF80050E079FC
:104E100038B1A06A4FF6FF71884202D2401CA062EE
:104E200000E0A562207B19270126012823D0022853
:104E300028D00F285AD0617821B12179884201D138
:104E4000FFF736FC206AE169884202D8206A401CDC
:104E50002062207801280DD0206AE169884209D3B8
:104E6000E069002806D0E0695649B0FBF1F0C007C0
:104E700075D0E6719FE060780028E3D0E07AFFF714
:104E8000A3FCDFE76846FFF72FFB9DF80010E07AF0
:104E9000FFF7D0FA00B1E07360780028D2D048481C
:104EA000E17A3430425C2274E27912B12574072928
:104EB00001D039B114E0A06A41F2883188420FD2A2
:104EC00080200CE0007858B9607A08B1212006E013
:104ED000207A08B1182002E0A07A08B17920207465
:104EE000207CC043C0B2FFF713FBABE725736078AB
:104EF000012804D1FFF7DCFBFF20FFF765FCE07A17
:104F0000401CC0B2E07208289CD3E572606A10B100
:104F1000606A401E6062606A002893D1627B52B171
:104F2000A069B0F5FA6F03D3A069B0F57A6F02D229
:104F3000A069401CA061E07BB0B3322152B9A27BD2
:104F4000824207D02562A5616162E2790AB92670C2
:104F5000E070E571152803D0132808D024E028E07C
:104F6000A269B2F5487F1FD12670E77019E0A369E6
:104F70001A22042B09D163783BB9A378012B04D101
:104F80002670E2702562A5616162A369B3F5C87FEE
:104F90000AD16378012B07D1A378012B04D12670A5
:104FA000E2702562A5616162A17B6173A073E57304
:104FB00048E72670E770207B401C20730020F8BD76
:104FC00004C107200070170004480021416181617D
:104FD00001224270817008467047000004C107201A
:104FE00070B56B494FF0FF354A79082A03D32E2854
:104FF00070D1082A6ED8664B34335C286BD020DC25
:10500000A0F12004362C52D2DFE804F09D5151511A
:10501000515151A75151AB51AFA151A96A5A888A38
:105020008C978699629B515151A351515158626C92
:10503000607A7C51665A51665C51516A70935897F8
:1050400080547E2870D011DCA0F15F04172C2ED282
:10505000DFE804F07B812D4A505456582D443A2DF8
:1050600042382D525A2D714E2D5C3200D0283DD041
:105070000DDCA0F1C004102C19D2DFE804F01F4DA4
:10508000294B1841181818181818182D3149EE28EE
:105090003AD006DCD12825D0D62846D0D72806D14C
:1050A00040E0EF2828D0F62841D0F7283AD02E2823
:1050B0005CD161E03E2059E01C2057E0772055E0AC
:1050C000062053E0382051E030204FE05F204DE0D3
:1050D0007F204BE059E044E0762047E0742045E033
:1050E0003F2043E0392041E07C203FE073203DE059
:1050F00050203BE0582039E0542037E05E2035E076
:10510000792033E0712031E05C202FE078202DE021
:1051100037202BE0312029E07D2027E05B2025E0AF
:105120004F2023E0662021E01DE0BE201EE09C20F1
:105130001CE0BF201AE0DC2018E06D2016E00720FC
:1051400014E06F2012E0002010E008200EE0402064
:105150000CE048200AE0202008E0022006E01020B1
:1051600004E0042002E0012000E080209854487907
:10517000401C4871002070BD3AB1521ED0B2487137
:105180001A5C42F080021A54F1E7284670BD000014
:1051900004C10720082802D34FF0FF3070470249AE
:1051A000487100207047000004C10720004A1047E2
:1051B000F11FFF1F534E0027FF203760B780B771E4
:1051C0007071FEF711FBFCF769FCFEF7F7FAFBF7CD
:1051D00039FCFFF7F9FEFCF7C5FE4B4885684B4CE0
:1051E000DFF82CB1DFF82C914FF4800A80460A20BA
:1051F000FFF794FBC0B2182826D0D8F80800411B4E
:105200005945F4D3606820F440506060606C20F42D
:10521000405040F400506064C9F81CA0D9F8001058
:1052200041F48001C9F80010FCF77CFEFBF71AF985
:10523000F0B300F0E7F9D8B30220FBF7E2F896F9F3
:105240000500401C3ED041E0606820F440506060A2
:10525000606C20F4405040F4005060644D46C9F842
:1052600018A0D9F8000040F48000C9F800002AA076
:10527000FBF720FC206920F440002061206D20F421
:10528000400020654FF40060E865286C20F4006061
:105290002864D8F808104046224A6B6D5B0503D598
:1052A00083685B1A9342F8D3696D4905BCD400E06A
:1052B0000FE0816842F2107283685B1A9342FBD35D
:1052C0007771B1E718488069FFF736FD01207070EB
:1052D00004E00220FBF795F87770777113A0FBF7D5
:1052E000E9FB0A20FFF71AFBC0B20F2808D14021C2
:1052F0001148FAF742FF4022D1010F48FEF712FA97
:10530000FFF724FBBCC007200000094000C002409A
:10531000400D030000C009202D2020202020202047
:105320000000000080C3C901005B00002020626F04
:105330006F74202000000000F9DB0720F0B50B306F
:10534000154D20F007010024144A0FE003688B423A
:105350000BD38B4205D95E1A43184768C3E900672F
:1053600000E04368136002C004E0021D10680028DA
:10537000ECD12046002802D1286808B10020F0BDF9
:10538000064A07481060074A121A22F00702C0E9CD
:10539000002401202860D7E764C1072060C10720EE
:1053A0000400001000600010FFB50246002002EB70
:1053B000420501464FF440566C4603AA6B1844F868
:1053C0002130B34202DD002004B0F0BD094F07EBED
:1053D0006307DB073F78575401D03B095354535CB4
:1053E0008F0003F00F035354BB40491C184403299A
:1053F000E4DBE9E781C10720084A32231360C2E9F0
:10540000010107484FF47A710068B0FBF1F0D060F9
:1054100002F114011046FFF7C9BE00003CDC072072
:1054200000C107202DE9F0471D4A00234FF4007703
:10543000156A4FF4FF79C5F30724DFF868A04FF42D
:10544000E05CDFF86480194E25E0B84216D21328DC
:105450000CD014280CD048450CD0A0F58072FF3A2F
:105460000AD03E2813D81AF8002011E0EAB20FE063
:1054700022460DE055220BE0AA2209E0604506D243
:1054800008EB0002A2F5805292F8002E00E0002204
:10549000F254401C5B1C8B42D7D3BDE8F087000060
:1054A00078C00720C05A000081C10720F9DB07201F
:1054B000FEB534A30D460ECB8DE80E003449496D80
:1054C000490521D4B0F5007F1ED3324B324CB0F5E4
:1054D000E05F1AD29968A269891A304A914204D3CE
:1054E0009968A1610021616061612D4A0021A2F5E6
:1054F000D05307E044181C44565CA4F58054491C62
:1055000084F8006EA942F5D3FEBD616921B999689E
:10551000A16199686161A060224949790029F3D1AC
:1055200099686269891A204A914224D21F4A01214E
:1055300011709968A16199686161A1686268411AF6
:1055400015489142406A02D9814200D26160C10887
:1055500060685F224030B0FBF1F16846FAF706FE62
:105560006846FBF7A7FA61682A460D4801F5005125
:10557000FEF7D8F8FEBD0EA0FBF79CFA0C20FAF758
:1055800040FFFEBD20204C4F416420200000000061
:1055900000C009200000094078C00720A086010053
:1055A00081DB0720BCC0072020A1070068C00720BE
:1055B0004C4F41642045727200000000FFB50DA6FB
:1055C0000446E1CE8DE8E100022902DA002004B0B1
:1055D000F0BD6018002100F8011D6946B3FBF2F52B
:1055E00002FB1535B3FBF2F34D5D00F8015DA042FF
:1055F000F4D8ECE73031323334353637383941427C
:105600004344454646F2044000210088A0F5194273
:10561000993A0AD04FF4C0404FF4002208C8904293
:105620001944FBD309B100207047012070470000E6
:1056300010B572B63324084B10C307C307484FF4A4
:105640007A710068B0FBF1F01860191D0248FFF78D
:10565000ADFD62B610BD00003CDC072000C1072094
:105660002DE9F041144C236803B920600020134D4C
:10567000636803E00F5C1E18401CAF559042F9D3DD
:1056800098184FF480766060B04212D12068FFF71E
:105690005FFB0A4D143D286800B1FEE7324607491A
:1056A0002068FFF7C5FF286800B1FEE700206060B2
:1056B00020600020BDE8F081C4C0072064DC072022
:1056C00000050F0A1B1E141133363C39282D2722E2
:1056D00063666C69787D777250555F5A4B4E4441D2
:1056E000C3C6CCC9D8DDD7D2F0F5FFFAEBEEE4E1C2
:1056F000A0A5AFAABBBEB4B193969C99888D8782B2
:1057000083868C89989D9792B0B5BFBAABAEA4A1A1
:10571000E0E5EFEAFBFEF4F1D3D6DCD9C8CDC7C291
:1057200040454F4A5B5E545173767C79686D676281
:1057300023262C29383D373210151F1A0B0E040171
:1057400003060C09181D171230353F3A2B2E242161
:1057500060656F6A7B7E747153565C59484D474251
:10576000C0C5CFCADBDED4D1F3F6FCF9E8EDE7E241
:10577000A3A6ACA9B8BDB7B290959F9A8B8E848131
:1057800080858F8A9B9E9491B3B6BCB9A8ADA7A221
:10579000E3E6ECE9F8FDF7F2D0D5DFDACBCEC4C111
:1057A00043464C49585D575270757F7A6B6E646101
:1057B00020252F2A3B3E343113161C19080D0702F1
:1057C00000002110422063308440A550C660E7707D
:1057D000088129914AA16BB18CC1ADD1CEE1EFF125
:1057E0003112100273325222B5529442F772D662CD
:1057F000399318837BB35AA3BDD39CC3FFF3DEE375
:105800006224433420040114E664C774A44485541C
:105810006AA54BB528850995EEE5CFF5ACC58DD5C4
:105820005336722611163006D776F6669556B4466C
:105830005BB77AA719973887DFF7FEE79DD7BCC714
:10584000C448E5588668A7784008611802282338BC
:10585000CCC9EDD98EE9AFF9488969990AA92BB964
:10586000F55AD44AB77A966A711A500A333A122A0C
:10587000FDDBDCCBBFFB9EEB799B588B3BBB1AABB4
:10588000A66C877CE44CC55C222C033C600C411C5C
:10589000AEED8FFDECCDCDDD2AAD0BBD688D499D04
:1058A000977EB66ED55EF44E133E322E511E700EAC
:1058B0009FFFBEEFDDDFFCCF1BBF3AAF599F788F54
:1058C0008891A981CAB1EBA10CD12DC14EF16FE134
:1058D0008010A100C230E32004502540467067606C
:1058E000B9839893FBA3DAB33DC31CD37FE35EF384
:1058F000B1029012F322D2323542145277625672BC
:10590000EAB5CBA5A89589856EF54FE52CD50DC5D3
:10591000E234C324A014810466744764245405440B
:10592000DBA7FAB79987B8975FE77EF71DC73CD723
:10593000D326F2369106B01657667676154634565B
:105940004CD96DC90EF92FE9C899E9898AB9ABA973
:105950004458654806782768C018E1088238A328AB
:105960007DCB5CDB3FEB1EFBF98BD89BBBAB9ABBC3
:10597000754A545A376A167AF10AD01AB32A923AFB
:105980002EFD0FED6CDD4DCDAABD8BADE89DC98D13
:10599000267C076C645C454CA23C832CE01CC10C4B
:1059A0001FEF3EFF5DCF7CDF9BAFBABFD98FF89F63
:1059B000176E367E554E745E932EB23ED10EF01E9B
:1059C000005EBCE2613FDD83C29C7E20A3FD1F41DF
:1059D0009DC3217FFCA2401E5F01E3BD3E6082DCCF
:1059E000237D9FC1421CFEA0E1BF5D0380DE3C62BF
:1059F000BEE0025CDF81633D7C22C09E1D43A1FFAF
:105A00004618FAA427799BC584DA3866E5BB59079E
:105A1000DB856739BAE406581947A5FB7826C49A8E
:105A2000653BD987045AB8E6A7F91B45C6987A247E
:105A3000F8A6441A99C7257B3A6486D85B05E7B96E
:105A40008CD2306EEDB3510F4E10F2AC2F7193CD5E
:105A5000114FADF3702ECC92D38D6F31B2EC0E504E
:105A6000AFF1134DCE90722C6D33D18F0C52B0EE3E
:105A7000326C8ED0530DEFB1F0AE4C1291CF2D732E
:105A8000CA947628ABF517490856B4EA6937D58B1E
:105A90005709EBB536688AD495CB2977F4AA48160E
:105AA000E9B7550B88D6346A2B7597C94A14F6A8FE
:105AB000742AC896154BA9F7B6E80A54D7896B35EE
:105AC000EB3C904D53444F53352E30000202010001
:105AD0000110000004F80C000100010000000000AB
:105AE00000000000000029EFBEADDE41544F4C2005
:105AF000465072696E7446415431322020200000B5
:105B00000000000000100000002000000030000035
:105B10000040000000500000006000000070000025
:105B2000008000000090000000A0000000B0000015
:105B300000C0000000D0000000E0000000F0000005
:105B4000000001000080010000000200008002004F
:105B50000000030000800300000004000080040037
:105B6000000005000080050000000600008006001F
:105B70000000070000800700FF0F0000FF1F00006B
:105B8000FF2F0000FF3F0000FF4F0000FF5F0000FD
:105B9000FF6F0000FF7F0000FF8F0000FF9F0000ED
:105BA000FFAF0000FFBF0000FFCF0000FFDF0000DD
:105BB000FFEF0000FFFF0000FF7F0100FFFF01007B
:105BC000FF7F0200FFFF0200FF7F0300FFFF0300D3
:105BD000FF7F0400FFFF0400FF7F0500FFFF0500BB
:105BE000FF7F0600FFFF0600FF7F0700FFFF0700A3
:105BF000120110010000004051C2031300010420F3
:105C0000480109022000010100803209040000025D
:105C100008065062070582024000000705020240A4
:105C2000000000040309041C03410054004F004C11
:105C30000020002000200020002000200020002064
:105C4000002000280346005000720069006E0074B6
:105C500000200046006C00610073006800200020F6
:105C600000200020002000200020001A03460069C8
:105C70000072006D00770061007200650030003036
:105C800000300030000E034D0065006D006F0072A3
:105C900000790000153B000000000000493C0000B6
:105CA00000000000000000000000000000000000F4
:105CB00000000000000000000000000000000000E4
:105CC00000000000000000000000000000000000D4
:105CD000000000000102040820100108F902000081
:105CE000F9020000D9070000FD070000D9070000F5
:105CF000FD070000FD070000FD070000B5070000DC
:105D0000F9020000F9020000D9070000FD070000B9
:105D1000D9070000FD070000FD070000FD07000097
:105D2000B5070000B5230000AD230000D52000001A
:105D3000D51F000011250000ED280000092C0000EF
:105D4000612C0000F9210000C1130000B91300000C
:105D5000E1110000D51F0000112500008116000090
:105D6000CD3300008517000011130000073000003C
:105D700001300000D5200000D51F000011250000D3
:105D80000D300000CD33000025340000F921000063
:105D90000000000000000000000000000000000003
:105DA00000000000000000000000000000000000F3
:105DB00000000000E45D000000C007206801000052
:105DC00008020000E45D0000000000100060000018
:105DD000484800000C5E000068C10720A0310000A8
:105DE00048480000BD41544F4C20465072696E74C3
:105DF000280548D4284B3D049EC0072043093D8414
:105E000001FFFF0210010545FFFFFFFF59777304F3
:105E10000480B27DBA799A19DA4E0608488D9D5CE5
:105E20005F2F14F78418C2C3A99EDB70723803EE8B
:105E300073258EA611A218B1581E44B0F8B2E428FA
:105E40004F1E3B72108C672E535DCA70900BA85288
:105E50009F9BB5569006701FE507566AB0D37A4BE4
:105E60007B00AEAD9328669C443E80B33E19CD07BF
:105E7000486B6535AE0DF5C1B15EF7DF4AD513212C
:105E80001145EA34EAAC98D78C96E4C8FB1B5CB4A5
:105E9000058BA3ED08FAEDD97E2959F98709DD11A3
:105EA0003FABBCBBC55FD67CFFD450824183B57687
:105EB000B9400D0E86840A2B2EB6EA2EF79694343E
:105EC000D024968CAD33B7165F27B3206FCB1C8AD6
:105ED0001EC641327987743493D0224B3189235CBA
:105EE000F16E382F3CE32D4783F6B2526878FE08F6
:105EF000A48D3F1CF816E7D2CE3FAF83D432050AFB
:105F0000D9F2A80B711B9C9FB60D86F2A1F8A95778
:105F1000DE6C1C736544B9F0273C5A39BB7872E8D3
:105F2000EBD5BCAFF672A18050BDE745C7894C5D8B
:105F30001D807C6E6CC37F1ED94223A24ABC6EDBDF
:105F40003816B3298AE34A5212943B6E0DE7E305F3
:105F50001845D0403C58B5F6DC9078A7907F587033
:105F6000DBC7026217FBEE551E52FCBA6D3D74048E
:105F7000E1082FD7287FEC0EF358FEA01222B3447D
:105F8000D267ED3602DBFF1F74FF6666BE795B46A3
:105F900034319CE52C8FB045D1ADA71818260A984E
:105FA000350D7E498061D0C5FE49A0E7476EAAA69F
:105FB000C4D045333F644D4467FD34FE53DEAB53DC
:105FC00054C6B21EC97BDB92FD237917435A9A7AD5
:105FD0004D3AB417219D411E4039EE86682526149E
:105FE0000C6A59B158D90BF26723CDDE9D401A488F
:105FF000B7ED3655AC1381F8CEAA9DF75FF95E0A6E
:00000001FF
